:020000020000FC
:1000000083CE00000000000020C0C2C194C00000E8
:1000100000009EC000000000000000000203040673
:10002000080C10182030406080000406080C1018DE
:100030002030406080A0C00000070F1F3F000D0D62
:100040000403060D0503030202004FB662FD0EC055
:10005000552009F00994C52DC095089483FDC795D6
:10006000C4BDC093A10064604FBE1895C0916400E8
:10007000089483FDC795C4BDC093A1006B7FC09158
:100080006400CF3F09F420C070FF02C082FD05C0AC
:100090004FBE939894989598189575FD0EC065FD80
:1000A0000CC0C091B300C0FD9298C1FDC298C2FDC2
:1000B000C198CAEFC095CA95F1F79398949895980E
:1000C0002092A1004FBE189524BCCC27C064C8BFA5
:1000D0006460F6CFC0CF70FFBECF65FDBCCF939AF2
:1000E000BACF70FFB8CF65FDB6CF949AB4CF70FF8A
:1000F000B2CF65FDB0CF959AAECF929A70FFABCFDD
:1001000065FDA9CFC7E0CA95F1F7939AA4CFC29A2B
:1001100070FFA1CF65FD9FCFC7E0CA95F1F7949A14
:100120009ACFC19A70FF97CF65FD95CFC7E0CA956A
:10013000F1F7959A90CF4FB6C9B7CF7EC9BF6E7F02
:10014000CCB5CE0DDDB5DF1DDBBDCABD4FBE1895EC
:100150003FB68F7EA9B7A072A2118061A9B7AF7D0B
:10016000A9BFA9B7AE7FA9BF7894A0916800AA23C0
:1001700041F085FD2BC0A0916800AA95A09368006E
:1001800025C040E050E085FD15C0A6B396FDA095C2
:10019000A0FD4FEFAEB5A06496FDAF7BAEBDAA2724
:1001A000A062A8BF8D7FA6B396FDA095A0FD5FEFCE
:1001B000451739F7A0E461FDA093680085FD03C0F1
:1001C000A0E4A093680040939700816085FD0EC075
:1001D000A0916900AA2331F0A0916900AA95A0938B
:1001E000690004C08061AA27A062A8BF80FF0AC07E
:1001F000A09197004A2F61FF8E7F85FD01C000C04E
:10020000409361004091B600443009F004C0A091D1
:100210006100A0936300A52DA03408F06860A09150
:100220006000A395A093600059F0F894A9B7A1606D
:10023000A9BF84FF03C0A9B7A062A9BF3FBE18959C
:10024000A0917400A395A093740042E050916800BF
:10025000552329F085FF03C05A9550936800A0915B
:100260009700A13018F020929A000DC020929B00B8
:100270002092A500A0919A00AF5FA0939A0018F079
:10028000AFEFA0939A00B09061005091B600523049
:1002900049F466FF91F0A2E3BA1678F0A0918700C6
:1002A000A0936100533049F466FF39F0A2E3BA1617
:1002B00020F0A091C200A0936100509162005B15F4
:1002C00021F010F05A9501C05395509362004A9561
:1002D000D1F65091A500539509F45A955093A50075
:1002E000A091A600AA95A093A60009F046C0A1E09F
:1002F000A093A60045E0A091A7005A17F0F1A091A5
:10030000A8005A1728F441E0A3E0A093A60007C074
:10031000A091A9005A1718F441E04093A600D0908C
:100320009D00C0906300DC14A8F0A091B600A4303A
:10033000D9F066FD0FC0C0929D00539511F0A091B9
:10034000A700A093A500A1E0A093A600ACE3A09312
:10035000620013C0A0919D00A40F20F45FEF5093A2
:100360009D0002C0A0939D00A0919D00AF3F29F485
:10037000AFEFA0939B00A093A500F894A9B7A1604C
:10038000A9BF84FF03C0A9B7A062A9BF3FBE18954B
:100390003FB646B557B58F7EA9B7A072A21180614E
:1003A000A9B7AF7DA9BFA9B7AE7FA9BF789481FDDA
:1003B00025C0AEB5AF7B96FDA064AEBD8260A6B38E
:1003C00096FDA095A0FF05C0409365005093660080
:1003D0001FC1AEB5A06496FDAF7BAEBDAA27A062DB
:1003E000A8BF8D7F85FF01C006C140E0A6B396FD82
:1003F000A095A0FD00C140939700EFC0AEB5A064EA
:1004000096FDAF7BAEBD8D7F61FF72C0AEB5AF7B99
:1004100096FDA064AEBDAA27A062A8BF82604093EB
:10042000920050939300A09090004A19B0909100D0
:100430005B09BB24A22C4C38520518F4209296007C
:1004400049C0A091D600AA2359F1483C520528F48E
:10045000A0E1BA2EAAE0AA2E23C04836A1E05A078E
:1004600028F4A8E0BA2EAFE0AA2E1AC0403DA2E0C0
:100470005A0728F4A4E0BA2EAEE1AA2E11C0403AE1
:10048000A5E05A0728F4A2E0BA2EACE3AA2E08C0D1
:100490004839A8E05A0720F4A1E0BA2EA8E7AA2E0E
:1004A000C42EA0919400CA1AD52EA0919500DA0A04
:1004B000DD202AF4AFEFC094D094CA1ADA0A209251
:1004C0009600A8E0A210A0E0CA14DA0618F4A1E091
:1004D000A093960040939400509395004091920011
:1004E00050919300409390005093910002E075C0AA
:1004F000A09165004A1BA09166005A0B94FD60C054
:1005000093FD5EC092FD5AC086FF03C0D52EC42E57
:100510000CC05695479591FD51C05695479590FD55
:100520004DC0D52EC42ED694C79461FD19C0AC2DF4
:10053000AC51AD2DA24008F005C0DD2089F4AC2DF2
:10054000A85C70F4A0916700A395AA2311F0A09372
:100550006700AA3008F44FC02092970081604BC01A
:10056000A0916700AA2319F0AA95A0936700A22C76
:100570005091BC0097FD02C0A090CA00AAEFAA0E3D
:10058000A22DA21DCA18DA0A4FB74170442319F0F0
:1005900040E050E015C0AFEFCA16D20418F04FEF9C
:1005A00050E00EC0A091AE00CA9E412D000C441F29
:1005B00050E008F012C04FEF50E00FC0569547953D
:1005C00094FF07C0552309F04FEFA42FA6954A0FBB
:1005D000521D4F3F520508F04FEF40939700816046
:1005E00061FF09C0AFE1A095A923AB299A2F8F7DA8
:1005F000BB2009F48062A0E4A093680085FF03C0DB
:10060000AAE0A093680061FD03C085FD01C08F7E54
:1006100085FD03C0A0E2A0936900F894A9B7A1608A
:10062000A9BF84FF03C0A9B7A062A9BF3FBE1895A8
:1006300011E00AC013E008C01AE006C01EE104C0C1
:1006400014E602C018EC00C005E1BB27BA95F1F72B
:100650000A95D9F71A95C1F708952AE338E709C032
:1006600020E33CE806C02AE234EB03C025E238EC84
:1006700000C012E095FD9F7D95FF9062BB27C29A56
:10068000BA95F1F7949ABA95F1F79498BA95F1F76B
:10069000C298BA95F1F7939AB091AF00BA95F1F775
:1006A0009398B7E8BA95F1F71A9521F7022FB22F70
:1006B000BA95F1F70A95D9F73A95D9F6C29A0895FD
:1006C000221B39E0001F3A9509F40895221F211BCF
:1006D00018F4210F8894F6CF0894F4CF622C722C72
:1006E000B0E08894B395221F331FE0F73795279524
:1006F0008894912E802E020B130B10F4192D082DC7
:1007000010F4889401C00894661C771CBA9571F7A0
:10071000172D062D0895322D11232AF43A950095B0
:100720001095031B130BF894029F712C002D129F40
:10073000912C802C7894780C172D921C292DB4E0E4
:100740006B2E2695179507956A94D9F7332321F0D8
:1007500000951095031B130B08950091B60004300B
:1007600009F474C0B0919700B95198F0B72FB670E2
:1007700081F466FD2BC005E09090C800B92DBA95B4
:1007800021F00AE0BA9509F002E1B0917B00B01BBC
:10079000E0F066FF0AC0B0919F00B0939D00BFEFEC
:1007A000B093A500B1E0B093A600B0916100B09302
:1007B000630020927F00209280002092810020928E
:1007C0008200209283006F7B41C060649090C800DB
:1007D000B92DBA9579F4B0916200B095BB1FBB1FDB
:1007E0001B2FB7950B2FB12FB170B3951B2FB02FC7
:1007F000BE7F25C0B92DBA95BA9581F4B09162003B
:10080000B095BB1FBB1FBB1F1B2FB7950B2FB12F65
:10081000B370B3951B2FB02FBC7F14C0B091620092
:10082000B095BB1FBB1FBB1FBB1F1B2FB7950B2F4B
:10083000B12FB770B395B3951B2FB02FB87FB054BD
:100840000B2F120900937F001093800008951091E0
:100850007B00169500917A000795B0917F00B01B40
:100860000B2FB0918000B10B1B2F28F40038BFEF85
:100870001B0740F009C00F37120508F405C00FE749
:1008800010E002C000E81FEF009384001093850081
:10089000089500918400B09181000B0F10918500A4
:1008A000B09182001B1F20E03091850033230AF4B1
:1008B0002A95B09183002B1F1AF4203F40F00AC004
:1008C0002F3008F407C00FEF1FEF2FE003C000E048
:1008D00010E020EF30916300B0919C003B1718F4BA
:1008E000323030F009C0B0918500BB235AF004C00B
:1008F000B0918500BB2332F40093810010938200F5
:100900002093830008952091D80000918400000F67
:1009100010918500111FFFDE11232AF40038BFEF6C
:100920001B0740F009C00F37120508F405C00FE798
:1009300010E002C000E81FEF002352F0B091620007
:10094000B01B0B2F18F0013008F00AC001E008C0FE
:1009500000950F5FB09162000B0F08F001C00FEF20
:100960000093860008952091D90000918200109193
:100970008300D1DE11232AF40130BFEF1B0740F0C2
:1009800009C00F3F120508F405C00FEF10E002C0C8
:1009900001E01FEF112352F0B0918600B01B0B2F26
:1009A00018F0013008F00AC001E008C000950F5FA0
:1009B000B09186000B0F08F001C00FEF00936300A9
:1009C00008950FEF677F71FD29C072FD09C068604F
:1009D000B0917B00BA3020F0B52DB03408F4677FB9
:1009E000B091D500BB23D1F0B0917B00BB23B1F017
:1009F0000FEF10917B0064DEF894B091730072FDEC
:100A0000B5E00B9F112D002D7894112309F00FEF05
:100A1000B0919F000B1710F400919F0000939E006F
:100A2000089500917A0010917B0000541140B0911C
:100A30009E0010F4BA9501C0B39511F0B0939E00DA
:100A4000089500D4B7E073FDB6E0B06CB7B9B6B1A5
:100A5000B068B064B6B9ECDDB7E073FDB6E0B06C79
:100A6000B7B9B6B1B068B064B6B9B6B1B6FDFDCF2E
:100A700004B115B1B6B1BF77B6B937D42AEB20931C
:100A8000AA00222309F441C030E03093AB00732E5A
:100A90007694622E6694620E731E262D372D0217F1
:100AA000130778F08090AA00BAEBB80DB093AA00B3
:100AB0008090AB00B0E0B81DB093AB00260D371DA1
:100AC000EECF8090AA009090AB001091AB001695ED
:100AD0000091AA0007951695079523E016950795AE
:100AE0002A95E1F72091B7002A9529F42092AA00CF
:100AF0002092AB000AC02A9521F0800E911E2A9503
:100B0000E1F78092AA009092AB0008952091B7007F
:100B1000B6B1B6FDFBCF04B115B1B6B1BF77B6B96A
:100B2000B091AC00B395B093AC00B83060F12092B6
:100B3000AC00B091D400BB2321F1112329F0B09176
:100B4000AD00BF3F61F009C0B091AD000B1739F0A7
:100B500020F4BB2321F0BA9502C0B395E1F30091D4
:100B60009C00B093AD00B93B50F400ECBA3A38F4B5
:100B700000E8BB3920F400E4BC3808F400E000933E
:100B80009C00777F08952130B1F00F3FB3E01B0741
:100B900090F4BAEBBB2379F0B091AA000B17B09197
:100BA000AB001B0740F4B0919C00BB2359F0BA95F1
:100BB000B0939C0007C0B0919C00BF3F19F0B39563
:100BC000B0939C0000919C00B0916300B01B10F4A6
:100BD00000916300B0919D000B1750F000919D00B3
:100BE000B0919D00BF3F21F0B0919D00B0939C005B
:100BF000502E00936400B091AC00B73009F47860D7
:100C0000089502E3F894B091DA000B9F012D000CD7
:100C1000001F7894B0919C000B1710F000919C007D
:100C20000093610000936300502E009364000093D2
:100C30009F00089520927A00B0EFB0937B00089552
:100C4000F8940CB51DB5209174007894309175001E
:100C5000609076000093750010937600031B1609D0
:100C600071FD03C076FD81C02BC07090770020938A
:100C700077002709222311F00FEF1FEF80907800F3
:100C80009090790030937800609279006918161975
:100C900010937C00009175001091760008191909D5
:100CA00020917A0030917B0036952795020F131F13
:100CB00010F40FEF1FEF00937A0010937B0029C010
:100CC00020917A0030917B003901B4E08B2EB2E0A4
:100CD0009B2E343010F08A949A94383010F08A9415
:100CE0009A94769467948A94E1F7261937099920A3
:100CF00021F0169507959A94E1F7200F311F209364
:100D00007A0030937B0028F43FEF30937A003093E1
:100D10007B00323008F4706471FF02C0B3E00DC094
:100D2000B091C60000917100023838F0B395003AD6
:100D300008F0B395B63008F0B5E09B2EB4E08B2EEA
:100D400010917B0000917A0024E0169507952A9572
:100D5000E1F70819120928F0B02FB250B12FB209EB
:100D600010F402E010E0980126C020917A00309142
:100D70007B0039017694679466946694669426198C
:100D8000320906950695200F321D20937A00309384
:100D90007B00323008F07F7B04E03695279536954E
:100DA000279526952695201B10F0223008F422E086
:100DB00089019090C60060FDFECFE0908C00F0901D
:100DC0008D006160B9B7B061B9BF380176FD44C02C
:100DD0007694679400938C0010938D00B92DB330F6
:100DE000E1F0B0FD04C0060D171D930106C0000F11
:100DF000111F0250120922E030E0B92DB33068F023
:100E000020938E0030938F00009388001093890008
:100E100060928A0070928B003DC000938E00109308
:100E20008F00209388003093890060928A0070922E
:100E30008B0071FF10C0B0916D00B33060F0009175
:100E40008F0010917C001595010F28F022F0209260
:100E50008E0000938F001EC0669400938C00B92D05
:100E6000B33091F0B0FD03C0060D262D03C0000F76
:100E7000025022E0B92DB33038F020938E00009359
:100E8000880060928A0006C000938E00209388003C
:100E900060928A0000917D0002FD0350013049F408
:100EA00095FD12C0B0B7B860B0BFB0E0B06CB7B9D4
:100EB0000EC0023039F4B0B7B860B0BFB1E0B06C6A
:100EC000B7B905C095FDEECFB0B7B77FB0BF009101
:100ED000A400000F10F4BBE60B270093A40060FDF4
:100EE000FECFB2E0B0936E006160B9B7B061B9BF38
:100EF000B72FB670A1F020917A0030917B00369523
:100F00002795F8940CB51DB5020F131F1BBD0ABD24
:100F10006160B0E1B8BFB9B7B061B9BF7894089566
:100F2000606120927E0020E067FD20E206C06061E3
:100F300020927E0020E267FD20E0789401E076FDBB
:100F400011C0B72FB67009F06F7EB0917B00B5501D
:100F500048F002E0B55020F003E0B55008F006E09C
:100F600071FD0AE060FD12C0B0917E00BB2371F0FC
:100F700071FF08C0B0916D00B33020F0B0916E00E9
:100F8000BA9519F4789470615EC0AEDF7894000071
:100F90000000F89476FD16C010917B00173008F021
:100FA00017E0B5E01B0F72FD10E183FF110F62FF28
:100FB000110F71FD12E8B4B56090A100B61990F25E
:100FC000B10B80F2B0B71B2FB77FB0BFB8B1B0B7CD
:100FD00013FDB860B0BFB0917E00B395B0937E00B2
:100FE000B8B176FD06C0B1E071FDB2E0BA95F1F797
:100FF000B8B1B072B21709F01BC071FF05C00395FC
:101000000A3008F00395AECF64FF97CF6F7E3CB5F2
:101010006DB470907A0080907B00370D681C6BBCBB
:101020003ABD6160B0E1B8BFB9B7B061B9BF85CFB3
:10103000B0916D00B23008F480CF64FD7ECF0A9588
:1010400009F090CF7F7E20918E0030918F00F89430
:10105000B0E1B8BF0CB51DB5020F131F1BBD0ABD13
:10106000E0908800F09089006160B9B7B061B9BFC5
:101070007894B72FB67039F0B0916D0072FFB395C8
:10108000B0936D0009C074FF07C067FD05C064FD23
:1010900003C0BF91BF91E7C4089500E063FF03C0A0
:1010A00064FF01C001E0F89410917100B7E01B9F4C
:1010B000212D102D7894200F26951795269517959C
:1010C0002695179510937100183718F4B8E7B09368
:1010D000710000917100B09172000B1720F06062F6
:1010E00093989498959860FDFECFE0908A00F090D8
:1010F0008B006160B9B7B061B9BF0895AC98B2E038
:1011000095FD07C0F894B0937D00C29A92987894A8
:10111000EAC0F894B0937D00C29AC1987894E3C075
:10112000AC9AB3E082FF24C095FD11C002E0F894B0
:10113000B0937D00E7E8F0E00093B3009598C19A82
:1011400062FF02C0949A01C0C2987894CCC002E0B9
:10115000F894B0937D00E7E8F0E00093B300939833
:10116000929A62FF02C0949A01C0C2987894BBC060
:1011700095FD0BC0F894B0937D00E1E7F0E0959801
:1011800062FF01C0949A7894AEC0F894B0937D0049
:10119000E1E7F0E0939862FF01C0949A7894A3C0CD
:1011A000AC98B4E095FD07C0F894B0937D00929A96
:1011B000C198789498C0F894B0937D00C19A9298A1
:1011C000789491C0AC9AB5E082FF24C095FD11C01F
:1011D00001E0F894B0937D00EDE7F0E00093B300F8
:1011E0009498C29A62FF02C0939A01C09298789430
:1011F0007AC004E0F894B0937D00E1E9F0E0009358
:10120000B3009498C29A62FF02C0959A01C0C19837
:10121000789469C095FD0BC0F894B0937D00EBE61F
:10122000F0E0949862FF01C0939A78945CC0F894BF
:10123000B0937D00E7E7F0E0949862FF01C0959AD3
:10124000789451C0AC98B6E095FD07C0F894B0937F
:101250007D00C19AC298789446C0F894B0937D00FE
:10126000929AC29878943FC0AC9AB1E082FF24C0B1
:1012700095FD11C004E0F894B0937D00E1E9F0E041
:101280000093B3009398929A62FF02C0959A01C0AE
:10129000C198789428C001E0F894B0937D00EDE700
:1012A000F0E00093B3009598C19A62FF02C0939A50
:1012B00001C09298789417C095FD0BC0F894B09334
:1012C0007D00E7E7F0E0939862FF01C0959A78947B
:1012D0000AC0F894B0937D00EBE6F0E0959862FFC9
:1012E00001C0939A78946F7D08952AE630E0F90161
:1012F0002092B300939894989598929AC29AC19A22
:101300006B7F0895A4EBB0E007E00D9307E00D9329
:1013100001E00D9304E00D930FEF0D930D9309E0A1
:101320000D9302E00D9301E00D9301E00D93A0EC0D
:10133000B0E001E00D9300E00D9304EB0D930FEF8F
:101340000D930D930D9303E00D930FEF0D9301E0BB
:101350000D930FEF0D9305E20D9300ED0D9308E74C
:101360000D9308EC0D9304E00D930FEF0D9301E046
:101370000D9300E00D930AE70D930AE00D9300E052
:101380000D9301E00D9300E00D930FEF0D93089581
:101390002091BB008B7F233009F48460B091BC00A6
:1013A0009F7DB1FD90629F7BB091BD00B1FD9064C7
:1013B000223011F0886001C0877F08950A95E00F00
:1013C000F21DB4910895ECE1F0E00091B400F6DF75
:1013D000B093D800ECE1F0E00091B500EFDFB093FE
:1013E000D900EAE2F0E00091BA00E8DFB093DA0059
:1013F0000091D300002309F40395013108F001E1C5
:10140000B02FB00FB00FB093A7001B2FB10FB10FCB
:10141000B00FB093A800B10FB00FB00FB093A900F8
:10142000B091D0000FEF1CE0B23011F400EA1AE0E6
:10143000B33011F402E815E00093720010937300CA
:10144000E8E3F0E00091D700B9DFB093A20008957F
:1014500008952091CA003091CB00B091BC00B33008
:1014600009F43E5097FF02C020E03FEFB32FB21BBC
:101470006B2EB25810F4B2E86B2E00E00395609E1C
:10148000B12DBD57D8F30093AE0008959068E1DF09
:10149000D5D820E030E0B0E16B2ECCD8B0919700E9
:1014A0002B0F321D6A94C9F7B4E036952795BA958B
:1014B000E1F7822E9F77CDDF0895F894E3E0F0E026
:1014C000B9E0B7BFB491B078C1F3F894A895B1B5BD
:1014D000B861B1BDB0E0B1BDB4E0BEBFBFE5BDBF56
:1014E00004DFB6E0B8BBB6E1B7BBB8E0B5BBBCE162
:1014F000B4BBB4E0B2BBBCE3B1BB2224A0E0B0E01B
:101500002D92AA31E9F7A0E6B0E00FEF2D920A95EF
:10151000E9F7B1E0B093A400F5DEDED2B7E0B06C3D
:10152000B7B9B6B1B460B068B6B90091CC00009359
:10153000AF00B1E0B0936A00F89484D88ED87ED81A
:101540008FD87CD890D87AD856D37CD87BD878D806
:10155000F8940AEF1AEFA6B396FDA095A0FF1FC05E
:101560001A95C9F70A95B1F7E0E0FCE1B591B43EF0
:1015700039F4B591B03E21F4B591BF3F09F40CC0E8
:10158000E0E0F395F395B591B83F49F4B591B439DE
:1015900031F4B591BA3A19F4EE27F6950994F8DECC
:1015A00012DF56DF56DF0091CC000093AF009DDEC6
:1015B000B2E0B3BFB2E0BEBDB2E0B5BDB1E5B8BF09
:1015C000B9BFB0B70B2FB77FB0BFB8B1B0B703FD8D
:1015D000B860B0BF2DD8789434DABEB5B06496FD4B
:1015E000BF7BBEBDB9B7B062B9BFBB27B062B8BFE1
:1015F0008D7F28D8626033E02CE0B0919600BB2349
:1016000021F42CE03A9509F4A3CF18D880FFA0CF9D
:101610008E7FB0919700B23078F3B92FBF710091EF
:10162000990000939800B0939900B01729F72A9574
:1016300021F76D7FBEB5B06496FDBF7BBEBDBB27F5
:10164000B062B8BF8D7FB091D600BB2321F4806219
:10165000B92FB0709B2F8F7B20926700F1D785FF49
:1016600005C0B0916700BA3008F08064E3D702E0AB
:1016700085FF01C000E0B0919700B017B8F3F8946F
:10168000ECD7EBD7EAD77894DDD720928700D2D772
:10169000B091C000B13008F46EC0B0916A00B130B2
:1016A00008F469C085FD18C0B0919700BF3F08F4E9
:1016B00062C0F894DBD77894C3D7B0919700B1306B
:1016C000C0F7F894CAD7B8D7C8D77894B9D7B0912B
:1016D0009700BF3FB0F3C1C2B8E09B2E9068F8946A
:1016E000B8DE7894ADD7F8949F77B3DE80909700FA
:1016F000B0919700BF37789408F445C099D7F89413
:10170000B5D778949A9451F7C1DEB82DB550B093FF
:10171000CB0098D7F8940DD273D27894BAE09B2E70
:101720009068F89496DE78948BD7F8949F7791DE42
:1017300080909700B0919700BF37789478F778D76A
:10174000F8948BD779D789D778949A9449F79EDE05
:10175000B82DBB5FB093CA0075D7F894EAD15FD2B9
:1017600078946ED7F89475DE7894B0919700BF3F67
:1017700008F498CF72C200919700B09187000B17C0
:1017800010F0009387005CD701E0B091BC00B3502B
:1017900009F405E0B0919700B01708F078CFF894FD
:1017A00065D764D763D778944DD720926A0020928A
:1017B0006B0020926C00B0916B00B395B0936B00FE
:1017C000BF3F69F5B0916C00B395B0936C00B091D8
:1017D000CE0009E1BA9559F002E3BA9541F00DE760
:1017E000BA9529F00AEFBA9511F020926C00B091E9
:1017F0006C00B017A0F0B0916C00BA95B0936C007B
:10180000B4EBB0936B00B091CD00B093AF00F894FF
:101810002DD77894B091CC00B093AF0011D70CD7EE
:10182000B0916800BB2319F485FF01C091CE01E09F
:1018300085FD01C006E0B0919700B01708F4BBCF5A
:10184000FFD6B0916800BB2309F482CEF8944DDD39
:10185000209261002092620020926300522C20921C
:1018600064002092A3007894B091B900BB0FB093AC
:10187000A00020927F002092800020928100209280
:101880008200209283002092AC0060E070E0209201
:101890007100B8E0B093AC007860CAD6B7E073FDD1
:1018A000B6E0B06CB7B9B6B1B068B064B6B9B6B1AD
:1018B000B6FDFDCF04B115B1B6B1BF77B6B91123EE
:1018C00009F00FEF0093AD0021D9B8E0B093AC0060
:1018D00078608090BB00B2E0B093BB0059DD80928D
:1018E000BB00F894BFEFB0939C008BD9B09161001E
:1018F000B0939C00B0939D00B0939E007894B1E0AB
:10190000B0936100B09363005B2EB0936400B0931A
:10191000A600B0919B00B093A500B091BC00B3307D
:1019200019F49F7D87FD90627160726020926D0056
:1019300089DC9ADC7FD984D97DD982D97BD906C04C
:10194000F89426DD78942092AC00777FF0DA05D702
:10195000A4DBD4DB75D9E4DA66FD79D776FF31D81C
:1019600076FD5FD89ADBDCDB6BD9E1DA66FD91D7D7
:1019700094DB16DC65D9D4DA66FDC5D78EDB22DCB4
:101980005FD9D5DA66FDEFD788DB5CDC59D9C8DAD8
:10199000B7E073FDB6E0B06CB7B9B6B1B068B0648B
:1019A000B6B97BDB61DC4CD9B1D871FF20C067FDD3
:1019B0001EC0B0919F00B0939C00B0939D00B09169
:1019C0009B00B093A500B1E0B093A60018E12CE015
:1019D000B0916D00B11728F07D7F746020936F0087
:1019E00006C0B0919700B13008F0B0CF46C072FF8A
:1019F00010C067FD0EC0B0916F00BA9511F47B7FE7
:101A00009FCFB0936F00B0919700B13008F09ECF98
:101A100034C020927000B0919A00B13058F0B0916B
:101A20009F00B0939D00B0919B00B093A500B1E0E2
:101A3000B093A600B0919A000AEFB01708F01DC04D
:101A400085FF04C0B0916800BB23B9F000EF67FFC9
:101A500005C0B0919F00B0939C0000E2B0917B0064
:101A6000B01708F473CFB0917000B395B0937000C5
:101A7000B0919700BB2309F002C020927000F89447
:101A800034DC8090BB00B2E0B093BB0081DC80927C
:101A9000BB00209261002092620020926300522CD1
:101AA000209264002092A0007E7F7894C1D51DDC36
:101AB000B7E0B06CB7B9B6B1B460B068B6B985FF7D
:101AC00005C0B0916800BB2309F442CDB091C100BC
:101AD000B13008F0CBCD6BCEEDE0F0E023D0053A8D
:101AE00009F01BC0EEE0F0E01DD00A3509F015C08A
:101AF0003AE0A4EBB0E0E3E0F0E014D00D933196CF
:101B00003A95D9F738E1A0ECB0E0EFE0F0E00AD088
:101B10000D9331963A95D9F702C0F4DB0AD0E7E28B
:101B2000F0E00895E199FECFEEBBFFBBE09A0DB364
:101B300008951ED03AE0A4EBB0E0E3E0F0E00D91B0
:101B40000FD031963A95D9F738E1A0ECB0E0EFE04C
:101B5000F0E00D9105D031963A95D9F712D008955D
:101B6000E199FECF0DBBEEBBFFBBE29AE19A08956F
:101B7000EDE0F0E00FEFF4DFEEE0F0E00FEFF0DF8C
:101B80000895EDE0F0E005EAEBDFEEE0F0E00AE5D5
:101B9000E7DF08953091B0000091B100313011F4C9
:101BA0000093B400323011F40093B500333011F4D7
:101BB0000093B600343011F40093C800353011F4AE
:101BC0000093B700363011F40093BA00373011F4A7
:101BD0000093C600383011F40093BB00393011F483
:101BE0000093D0003A3011F40093BC003B3011F464
:101BF0000093BD00089525E025D52A95E9F70895BD
:101C00002CD52ED530D532D517D527D529D52BD5DE
:101C10002DD512D522D524D526D528D5089526D55B
:101C200022D51ED51AD508D521D51DD519D515D53E
:101C300003D51CD518D514D510D508958090B000C3
:101C40009090B1000AD509D508D5F6D48A94D1F779
:101C50000DD5F2D49A94E1F70895F894D1DF7894F1
:101C6000CADFC9DFB1E0B093B000B1E0B093B1001A
:101C70002092B200F894E2DF7894B5E06B2E709079
:101C80009700E0D4B09197007B16C9F7B13018F0F7
:101C9000BF3F40F107C07EDFF8944BDFB1DFB8E013
:101CA000B1BDA9DF6A9459F7B091B200B395B09372
:101CB000B200B33008F4DECF9EDFB091B100B3952F
:101CC000B093B100F894B091B000BA95EEE3F0E0B3
:101CD000EB0FF21D049178940395B091B100B01709
:101CE00008F4C6CF88DF87DFB091B000B395B0931A
:101CF000B000B091B000BC3008F4B7CF03DBF8946B
:0A1D000018DFB8E0B1BD77DFD8CBE3
:00000001FF
